:100000000C94340018950000189500001895000015
:10001000189500000C94D202189500001895000065
:10002000189500001895000018950000189500001C
:10003000189500000C94C204189500001895000053
:1000400018950000189500001895000018950000FC
:1000500018950000189500001895000018950000EC
:1000600018950000189500008FEF8DBFC8EDE6E9E8
:100070004E2E84E08EBFD4E0F4E05F2EA89584B7C6
:10008000082E877F84BF88E1992780936000909332
:100090006000EEEFF3E0A0E0B1E088278D933197A8
:1000A000E9F76624219A259874B7777F74BF88E1B1
:1000B0008093600080E0809360002D9A7FE07093D1
:1000C0006D00789480916000886180936000877FE4
:1000D000809360000E943503A0E0B1E00C93009192
:1000E0000001003111F40C949402009100010030E1
:1000F00011F00C94800081E0809300010C940501C4
:10010000013011F00C94890082E0809300010C947E
:100110000501023011F00C94920083E080930001FD
:100120000C940501033011F00C949B008CE080933B
:1001300000010C940501043011F00C94A40084E03B
:10014000809300010C940501053011F00C94AD0072
:1001500085E0809300010C940501063011F00C94A9
:10016000B60086E0809300010C940501073011F081
:100170000C94BF008DE0809300010C9405010830C1
:1001800011F00C94C80087E0809300010C940501E5
:10019000093011F00C94D10088E0809300010C9498
:1001A00005010A3011F00C94DA0089E08093000117
:1001B0000C9405010B3011F00C94E3008EE0809359
:1001C00000010C9405010C3011F00C94EC008AE055
:1001D000809300010C9405010D3011F00C94F50092
:1001E00080E0809300010C9405010E3011F00C9416
:1001F000FE008BE0809300010C9405010F3011F09C
:100200000C9405018FE0809300011D9B0C94230149
:1002100070916800746070936800219A81E88093FF
:10022000800081E080938100A0E0B1E00C910A930E
:1002300080E69AEE0E949D04709168007B7F709327
:1002400068000C9494027091680074607093680068
:10025000219A80E48093800089E08093810000915E
:100260000001003011F00C9447015A924A92D201D9
:10027000EAE7FAE00E948F0484E00E9477030E947C
:100280009602229684E00E9418030C948F0201309B
:1002900011F00C945D015A924A92D201EEE7FAE015
:1002A0000E948F0484E00E9477030E9496022296A7
:1002B00084E00E9418030C948F02023011F00C9419
:1002C00073015A924A92D201E2E8FAE00E948F0446
:1002D00084E00E9477030E949602229684E00E94A6
:1002E00018030C948F02033011F00C9489015A9278
:1002F0004A92D201E6E8FAE00E948F0484E00E946C
:1003000077030E949602229684E00E9418030C94C0
:100310008F02043011F00C949F015A924A92D2013C
:10032000EAE8FAE00E948F0484E00E9477030E94CA
:100330009602229684E00E9418030C948F020530E6
:1003400011F00C94B5015A924A92D201EEE8FAE00B
:100350000E948F0484E00E9477030E9496022296F6
:1003600084E00E9418030C948F02063011F00C9464
:10037000CB015A924A92D201E2E9FAE00E948F043C
:1003800084E00E9477030E949602229684E00E94F5
:1003900018030C948F02073011F00C94E1015A926B
:1003A0004A92D201E6E9FAE00E948F0484E00E94BA
:1003B00077030E949602229684E00E9418030C9410
:1003C0008F02083011F00C94F7015A924A92D20130
:1003D000EAE9FAE00E948F0484E00E9477030E9419
:1003E0009602229684E00E9418030C948F02093032
:1003F00011F00C940D025A924A92D201EEE9FAE001
:100400000E948F0484E00E9477030E949602229645
:1004100084E00E9418030C948F020A3011F00C94AF
:1004200023025A924A92D201E2EAFAE00E948F0431
:1004300084E00E9477030E949602229684E00E9444
:1004400018030C948F020B3011F00C9439025A925D
:100450004A92D201E6EAFAE00E948F0484E00E9408
:1004600077030E949602229684E00E9418030C945F
:100470008F020C3011F00C944F025A924A92D20122
:10048000EAEAFAE00E948F0484E00E9477030E9467
:100490009602229684E00E9418030C948F020D307D
:1004A00011F00C9465025A924A92D201EEEAFAE0F7
:1004B0000E948F0484E00E9477030E949602229695
:1004C00084E00E9418030C948F020E3011F00C94FB
:1004D0007B025A924A92D201E2EBFAE00E948F0428
:1004E00084E00E9477030E949602229684E00E9494
:1004F00018030C948F020F3011F00C948F025A9253
:100500004A92D201E6EBFAE00E948F0484E00E9456
:1005100077030E949602229684E00E94180370914D
:1005200068007B7F709368000C946A0084E00E94EE
:10053000710382E00E947103EAEBFAE00E948204F8
:10054000EC81FD810E94AF030E944404EDE0F0E0E5
:10055000AA81BB810E949704EA81FB810E94B403B7
:10056000EEEBFAE00E9479040E94EE03EDE0F0E089
:10057000AA81BB810E949704EA81FB810E947B03D0
:10058000A881B981DD92EC92A881B9818D919C916D
:10059000909389008093880086E0481A80E0580A8A
:1005A000249608950F921F922F923F924F925F923E
:1005B0007F92AF92BF920F931F932F933F934F93CE
:1005C0005F936F937F938F939F93AF93BF93CF93DB
:1005D000DF93EF93FF938FB78F9309B10F3011F033
:1005E0000C94F702809160008860809360008F9186
:1005F0008FBFFF91EF91DF91CF91BF91AF919F910D
:100600008F917F916F915F914F913F912F911F91AA
:100610000F91BF90AF907F905F904F903F902F9041
:100620001F900F901895F894FFCF481A590A089513
:10063000481A8827580A0895AE7B9E5BAE5BC15B63
:100640009E65AE65C1659E6FAE6FC16F9E7BC17BBF
:10065000D55BD565D56FD57B3197F1F70895689453
:1006600062F80895E89462F8089500E18FEF8BB97D
:100670008FE08AB980EF8BB98EE18A95F1F74C9BB8
:1006800000E04D9B04E04E9B08E04F9B0CE080EFA8
:100690008AB98FE08BB98EE18A95F1F78827489B5C
:1006A00080E0499B81E04A9B82E04B9B83E0080FFE
:1006B0008AE090E00E945D030895EF93FF93EE2798
:1006C000E82BE92B31F0E8EEF3E03197F1F70197F1
:1006D000D1F7FF91EF9108955A924A92480E591E10
:1006E00008955A924A92480E8827581E0895480E37
:1006F0008827581E089533D0992711278F2D880FEA
:1007000080E8F82A802F881F08F41FEF41F08F57E8
:10071000082F07FD04C0003240F08FEF01C088278A
:10072000982FD82EE82EF82E09C08FE1801B082FB5
:10073000F694E794D79497950A95D1F7112351F041
:100740009095D094E094F09481E0980F8827D81E7B
:10075000E81EF81E0F2DFE2CED2CD92E0895D190F9
:10076000E190F19001910895219131914191519140
:100770000895102F90E8FF0C001F0927990FF79498
:100780001078652F90E8440F551F5927990F47950A
:10079000607800380895FF0C90E89027110F979526
:1007A000F794092F0895502F2D2D3E2D4F2D612F99
:1007B00008952DEC3CEC4CEC5DE366270FC0CFDFD9
:1007C000F2DFDD24EE2490E8F92E0FE307C0CCDF42
:1007D00005C02227332740E251E46627552351F113
:1007E000002381F1C6DF71F1162700585058089494
:1007F000050B18F407FD03C025C007FD23C046956F
:1008000037952795F694E794D79422D0FF202AF0C5
:10081000DD0CEE1CFF1C015073F09D2D969548F0E9
:10082000DD203AF4EE202AF491E0D90E9927E91E52
:10083000F91EB1CF07C09FE7092FF92A9FEFD92EE4
:10084000E92E0895DD24EE24FF24002711270895C2
:100850009F929924AA24BB2488E1D216E306F406C9
:1008600028F0D21AE30AF40A089401C08894991C6B
:10087000AA1CBB1CDD0CEE1CFF1C8A9571F7D92C41
:10088000EA2CFB2C9F90089574DFE1F25038D1F2EE
:100890001627005850580894051F12F418F4CBCFAF
:1008A00008F0D0CF0BD0FF202AF0BB0CDD1CEE1CD3
:1008B000FF1C71CF0F5F0BF4BECF6DCF9F929924B9
:1008C000AA24BB24992788E1990CAA1CBB1CDD1C17
:1008D000EE1CFF1C30F4920EA31EB41ED91EE91E9E
:1008E000F91E8A9589F79F900895C8953196002042
:1008F0000895FBDFD02CF9DFE02CF7DFF02CF5DFDB
:10090000002D0895F2DF202DF0DF302DEEDF402D99
:10091000ECDF502D089591E005C092E003C094E013
:1009200001C098E0E2DF0D929A95E1F7089594E016
:1009300081918D939A95E1F708958F939F93442722
:100940005527222733270991000FE8E3F6E0E00F4F
:100950000027F01F0E947504A02C0E947504902CA3
:1009600070916F00716070936F009F918F910E94E2
:100970005D0370916F007E7F70936F008827809376
:10098000810008958F938FB78F93EF93FF930F920A
:10099000042F152F490D8827581F1CD0702D022FAA
:1009A000132F2A0D8827381F15D0602D82E0680F7D
:1009B00066956695061A602D882780938900872F93
:1009C000860F809388000F90FF91EF918F918FBFDA
:1009D0008F9118958FE018230C5F1F4F1695079580
:1009E00016950795169507950F77EAEFF9E0E00F52
:1009F0008827F81F0E9475040895404346494C4FCC
:100A00005255585B5E606366686A6D6F7173757688
:100A100078797B7C7D7E7E7F7F7F7F7F7F7F7E7E00
:100A20007D7C7B7978767573716F6D6A68666360BB
:100A30005E5B5855524F4C494643403C3936333043
:100A40002D2A2724211F1C19171512100E0C0A0914
:100A5000070604030201010000000000000001017C
:100A60000203040607090A0C0E10121517191C1FA1
:100A70002124272A2D303336393C000086420000DD
:100A80009A420000A5420000B1420000B7420000B7
:100A9000C8420000CF420000F64200800843CD4C1F
:100AA0000D4300802543008037430080474300808A
:100AB0004B4300804E4333B35243000000400024B8
:020AC000744A76
:00000001FF
